:104DEB000000090101240200000301FA0400FA0586
:104DFB0000020A0A5A0B000F0C00FA0D00030E00FA
:104E0B00030F0132100096120132130AFA14010239
:104E1B0015000217010A18010A1905321A010A1B9B
:104E2B00010A1C053223011E2400642A00FA2B0000
:104E3B00FA2C50782D003C2E00462F001E300064BB
:104E4B003250783300003432FA350164360164375E
:104E5B000150380A643C00643E003C3F000140FFB7
:104E6B00FF411450420A5A430AC8440532450078A0
:104E7B004600FA4701224802034C00FA4EFFFF504E
:104E8B000606510596520A32530B28540A965601C0
:104E9B0002570546580002590A465A32FA5B010A74
:104EAB005C0A325E000A5F00FE61FFFF640210675E
:104EBB0001036A0A3C6B00006C329678013279016F
:104ECB0032FAFAFA0000090101240200000301FA88
:104EDB000400FA0500020A0A5A0B000F0C00FA0D27
:104EEB0000030E00030F0132100096120132130A59
:104EFB00FA14010215000017010A18010A190532EC
:104F0B001A010A1B010A1C053223011E2400642A04
:104F1B0000FA2B00FA2C50782D003C2E00462F0067
:104F2B001E3000643250783300003432FA3501649D
:104F3B00360164370150380A643C00643E003C3F44
:104F4B00000140FFFF411450420A5A430AC844056E
:104F5B00324500784600FA4701224802024C00FA1B
:104F6B004EFFFF500606510596520A32530B28543A
:104F7B000A96560101570546580001590A465A32FE
:104F8B00FA5B010A5C0A325E000A5F00FE61FFFFFA
:104F9B006402106701036A0A3C6B00006C3296785E
:104FAB000132790132FAFAFA0065006F0079008359
:104FBB00008D009700A100AC00B600C000CA00D461
:104FCB0000DE00E800F2005B0063006A0072007A0A
:104FDB00008200890091009900A100A800B000B8E0
:104FEB0000BF00C700CF00D600DF00E600EE00F6E2
:104FFB0000400046004C00520059005F0065006BFA
:10500B0000710077007D00830089008F0095009C64
:10501B0000A200A800AE00B400BA00C000C600CCCD
:0C502B0000D200D900DF00E500EB00F12E
:10009E00AE33AF34740A8E048F05FF1252A38C3523
:1000AE008D36AE33AF34740A8E048F05FF1252DCD8
:1000BE008C338D34E53445336013740AC39534FFA5
:1000CE00E49533FE8E338F34783512531EE550A8E7
:1000DE0035B80015D395364010E550C39536FFE47C
:1000EE009535FE8E358F368010E5502424C3953617
:1000FE00FFE49535FE8E358F36AE35AF3674236FF1
:10010E004E600674246F4E701AAE35AF3674236F80
:10011E004E70057550018003755002753622753587
:10012E0000800375500022900085E0B40104C20BDC
:10013E008002D20B900086E0B40104C20C8002D281
:10014E000C9000C3E075F0DCA4FFAEF0740A8E04D0
:10015E008F05FF1252A39007ABECF0A3EDF0A208AF
:10016E00401674038C068D071252C174011252B3DD
:10017E009007A9EEF0A3EFF07E017F00900081E0E2
:10018E001252C19000C4E08E048F05FF1252A37468
:10019E000AFF1252A38D399000CDE075F0DCA4FF5A
:1001AE00AEF0740A8E048F05FF1252A39007AFECC7
:1001BE00F0A3EDF09000CFE060139000CFE0F5F0EB
:1001CE00741684FF7E00EF9007B7F080067464907B
:1001DE0007B7F09000D7E0B4020674029000B9F0B1
:1001EE009000C9E0B402089000D7E064016002807C
:1001FE000674009000D7F09000D7E0B4010890008C
:10020E00ABE064026002800674019000ABF09000D7
:10021E00AEE0B40B0874E390006FF080499000AE2E
:10022E00E0B419129000C4E0904F9E12008CE4933B
:10023E0090006FF080309000AEE0B41E129000C4BB
:10024E00E0904FBC12008CE49390006FF0801790FA
:10025E0000AEE0B428109000C4E0904FE612008C7F
:10026E00E49390006FF090004BE0C394055022741D
:10027E00019000C7F09000C9E0B40206740190002E
:10028E00C9F09000B9E0D39402400674029000B910
:10029E00F09000E1E0B40117900024740FF0A37405
:1002AE00FFF0900026E4F0A3F074029000E1F090CD
:1002BE0000E1E0B40341900026E0FEA3E0FF9000D1
:1002CE0024E0FCA3E0FD12531674101252C1740800
:1002DE001252B3EF90006CF0EF700674FF90006C4A
:1002EE00F074009000E1F0900025E090006DF09029
:1002FE000024E090006EF0900072E0900034F090D8
:10030E000034E0240C900035F0900034E024189076
:10031E000036F0900035E0D39424400B900035E089
:10032E00C39424900035F0900036E0D39424400B13
:10033E00900036E0C39424900036F090003AE4F03A
:10034E00900034E064236007900034E0B4242090E1
:10035E000034E0B42306740290003AF0900034E0CA
:10036E00B4240690003A7401F09000347401F090B9
:10037E00003BE4F0900035E064236007900035E028
:10038E00B42420900035E0B42306740290003BF0B4
:10039E00900035E0B4240690003B7401F0900035D7
:1003AE007401F090003CE4F0900036E064236007A6
:1003BE00900036E0B42420900036E0B42306740298
:1003CE0090003CF0900036E0B4240690003C74019E
:1003DE00F09000367401F0900072E0FE9000D5E0CF
:1003EE002E90003EF09000B0E0B4016090003EE030
:1003FE006412600790003EE0B4240690003EE004D4
:10040E00F090003EE06411600790003EE0B42306D9
:10041E0090003EE014F090003EE0D39424400B9008
:10042E00003EE0C3942490003EF090003EE0D39452
:10043E0012400D90003EE0C3941290003FF0800AEF
:10044E0090003EE0241290003FF0807690003EE057
:10045E00640C600F90003EE06418600790003EE070
:10046E00B4240690003EE004F090003EE0640B6081
:10047E000F90003EE06417600790003EE0B4230644
:10048E0090003EE014F090003EE0D39424400B9098
:10049E00003EE0C3942490003EF090003EE0D394E2
:1004AE000C400B90003EE0C3940C90003EF0900088
:1004BE003EE0D3940C400B90003EE0C3940C9000B1
:1004CE003EF09000B8E0900037F0900037E0640BFB
:1004DE006007900037E0B41706900037E014F090F4
:1004EE000037E0640C6007900037E0B41806900007
:1004FE0037E004F0900037E0240C900038F09000C4
:10050E0037E02418900039F0900038E0D39424405E
:10051E000B900038E0C39424900038F0900039E03E
:10052E00D39424400B900039E0C39424900039F00A
:10053E0022C293C294C291C292C287C290E5B554B0
:10054E00EFF5B5E5B554DFF5B5C296C295C2A0C2BA
:10055E0097C2A2C2A1E5B554BFF5B5E5B5547FF576
:10056E00B5E5B554FBF5B5C20D7537469000BBE049
:10057E007005754902800375490390000C74FFF0F5
:10058E00A374DCF090009CE0900012F8E4F0E8A375
:10059E00F0C213C215C21774C8900028F074C89028
:1005AE00002CF074C8900030F0752600752500C23E
:1005BE0008756C00E54BB40903754B00753C009053
:1005CE00001AE4F0A3F0754C1E752800752700C2C2
:1005DE0010C211C2129007ABE0FEA3E0FF7403122B
:1005EE0052C174011252B39007A9EEF0A3EFF0C2FC
:1005FE0003900010E4F0A3F0C222900070E4F02209
:10060E0085F95085FA517E017F00E5511252C1E500
:10061E00502FFF50010E8E338F349007ABE0FCA3AA
:10062E00E0FDEF2DFDEE3CFC8C358D36E536F5FB11
:10063E00E535F5FC22053D22A2D8B34006C296C28E
:10064E0095C2A075D8402285A74F75A7109000B906
:10065E00E0640360079000D7E0B4022CA2D8B34048
:10066E0002C293A2D9B34002C294A2DAB34002C22C
:10067E0091A2DBB34002C292A2DCB34002C287A2B7
:10068E00DDB34002C290801BA2D8B34004C293C215
:10069E0092A2D9B34004C294C287A2DAB34004C274
:1006AE0091C29075D840854FA722900047E493647D
:1006BE0006600280FE74C89007B1F8E4F0E8A3F07B
:1006CE0075B50075840175A70075FF8075EF0690EE
:1006DE00003DE4F075C91075A70F75A1C775A70089
:1006EE0075D90075CE0C75A70F75F1FE75F2FF75F5
:1006FE00F30775F47875A4BA75A5FF75A60775AEE0
:10070E000075AFFF75D48175D5FF75D6FF75D7FF10
:10071E0075A70075A20175A14775F80975D8007502
:10072E00D90475DA0975D84075A71075D80075D932
:10073E000475DA0975DB0975DC0975DD0975DE09E5
:10074E0075DF0975D84075A70075E60875E7107551
:10075E00BC0175BE0475BD6C75BE0775BDA075BEBA
:10076E000875BD0175BC0075BB1875BC2075BA083F
:10077E0075E88075D11375B50075A70F75E1057510
:10078E00E20075C740C293C294C291C292C287C2A0
:10079E0090E5B554EFF5B5E5B554DFF5B5C296C2A3
:1007AE0095C2A0C297C2A2C2A1E5B554BFF5B5E5E8
:1007BE00B5547FF5B5E5B554FBF5B575970075974E
:1007CE0080740A1252937597C0E597542070028078
:1007DE00F8758F0275A700D2AF75980075A90C75C4
:1007EE00A70F75AB4375ADFB75AC1E75A71075C91C
:1007FE001875CA0075CB0075C80475A700758912E7
:10080E00758E04758C00758A00C2A9D28C758D0008
:10081E00758B00D2ABD28E75D9447532007531000E
:10082E00752E00752D00754600754700C29974C867
:10083E00F5097508001231F775B50074639007B1AC
:10084E00F8E4F0E8A3F01234837464F50975080037
:10085E001231F7C21E90005AE0B40108A2B5400250
:10086E00D21E802E90005AE0B4021175A70F75F3B8
:10087E000F75A700A2A34002D21E801690005AE068
:10088E00B4030F75A70F75F31775A700A2A4400246
:10089E00D21EA21EB3500302098E74089007B1F83F
:1008AE00E4F0E8A3F01233527464F50975080012EF
:1008BE0031F774099007B1F8E4F0E8A3F01233525F
:1008CE007464F5097508001231F7740A9007B1F8CF
:1008DE00E4F0E8A3F01233527464F50975080012BF
:1008EE0031F7740B9007B1F8E4F0E8A3F01233522D
:1008FE007464F5097508001231F7740C9007B1F89D
:10090E00E4F0E8A3F01233527464F509750800128E
:10091E0031F7740D9007B1F8E4F0E8A3F0123352FA
:10092E007464F5097508001231F7740E9007B1F86A
:10093E00E4F0E8A3F01233527464F509750800125E
:10094E0031F774029000BAF090005AE090007EF0F9
:10095E0090005AE0B401087400900086F0801C905C
:10096E00005AE0B4020874009000C9F0800D9000A7
:10097E005AE0B4030674009000D6F0D21A020A6E42
:10098E009007B1E4F0A304F01233527464F50975C4
:10099E0008001231F774029007B1F8E4F0E8A3F002
:1009AE001233527464F5097508001231F77403900E
:1009BE0007B1F8E4F0E8A3F01233527464F5097548
:1009CE0008001231F774049007B1F8E4F0E8A3F0D0
:1009DE001233527464F5097508001231F7740590DC
:1009EE0007B1F8E4F0E8A3F01233527464F5097518
:1009FE0008001231F774069007B1F8E4F0E8A3F09E
:100A0E001233527464F5097508001231F7740790A9
:100A1E0007B1F8E4F0E8A3F01233527464F50975E7
:100A2E0008001231F774019000BAF090005AE0906D
:100A3E00007EF090005AE0B401087400900086F039
:100A4E00801C90005AE0B4020874009000C9F08037
:100A5E000D90005AE0B4030674009000D6F0C21A4E
:100A6E001235F79000C4E07006740A9000C4F0903E
:100A7E00006FE0700674E390006FF0120135E5B57B
:100A8E004401F5B57406900049F0740190004AF0E7
:100A9E00740390004CF0740490004DF074189000A4
:100AAE004EF0740590004FF090004BE0B4040674C5
:100ABE000490004FF07406900050F07400900055B2
:100ACE00F07400900056F07401900057F07400908E
:100ADE000058F074FF900059F07433900148F07490
:100AEE0036900149F0742D90014AF0743290014B0A
:100AFE00F0742090014CF0743290014DF0744A90D5
:100B0E00014EF0745A90014FF07456900150F074EB
:100B1E0056900151F07454900152F0744990015363
:100B2E00F07420900154F07436900155F074439097
:100B3E000156F09000E0E090006CF0900097E0908D
:100B4E00006DF0900098E090006EF0C213C215C2D6
:100B5E001774C8900028F074C890002CF074C890D8
:100B6E000030F0C210C211C212A2B6B39209A2B3E3
:100B7E00B3920A752600752500753746754C1E9082
:100B8E000068E4F075271975286490000C74FFF066
:100B9E00A374DCF0C20D754B00C208752A007529CE
:100BAE0000900010E4F0A3F0743A900771F074FD19
:100BBE00900772F0756D00900069E4F0752C007569
:100BCE002B00900014E4F0A3F090009CE090001233
:100BDE00F8E4F0E8A3F090007DE075F032A4FFAEEB
:100BEE00F0900022EEF0A3EFF09007ABE0FEA3E052
:100BFE00FF74031252C174011252B39007A9EEF0A2
:100C0E00A3EFF0754A01900045E4F0C222C21F75B1
:100C1E006C00753C00C20EC20FC223C203754D009C
:100C2E00C204D205C206D207C21BC21CD21D74FE5C
:100C3E00900040F074FE900041F0C220D22190004E
:100C4E0070E4F0753800754400753A00753E3275E3
:100C5E003F00754000743C900043F0754100743CB9
:100C6E00900044F075420075430090001AE4F0A322
:100C7E00F0754500D2B2D2A4D2B0D2B1D2A3D2A7CF
:100C8E00D2A6D2A5D2B790007DE0D394FA400674D6
:100C9E00FA90007DF07E017F0090006EE01252C14E
:100CAE0090006DE02FFF50010E900024EEF0A3EFA8
:100CBE00F0EFD394FFEE940F4007900024E4F0A3DE
:100CCE00F090006CE0700674FF90006CF09000BA2B
:100CDE00E0D39402400674019000BAF09000BBE09D
:100CEE00700575490280037549039000BCE0D394EA
:100CFE0001400674009000BCF09000C2E0C3940A5C
:100D0E005006740A9000C2F09000CCE07006740198
:100D1E009000CCF09000CCE0B4FF0674FE9000CCB6
:100D2E00F09000D3E0D394FE400674FE9000D3F012
:100D3E0074019000D9F074019000DAF07400900004
:100D4E00DCF074009000E1F0D29CD2EC75CF01A2E1
:100D5E0098B35003021168C298E54764046006E533
:100D6E009964FF6002802AA2204004D2208020E5F0
:100D7E0047600874E62547900045F0754700E54644
:100D8E00600874F02546900045F0754600C220803C
:100D9E0002C220E5476003020E43754700E599B491
:100DAE00FF03754601E599B4FE03754602E599B455
:100DBE00FD03754603E599B4FC03754604E599B445
:100DCE00FA03754605E599B4FB03754701E599B439
:100DDE00F903754704E599D394E54007E599C39463
:100DEE00F0400280168599487547027E017F00E526
:100DFE0048C394E61252C18E2F8F30753200753172
:100E0E0000E599D394C74007E599C394E640028064
:100E1E001F85994875470374E5C39548F530752FBE
:100E2E0000AE2FAF3090503712528278311252FCF2
:100E3E00D299021168E547B401028003020F1BAE7E
:100E4E0031AF329000711252E8E599F078311253B9
:100E5E001EAE31AF32EFB40106EEB40702800302CC
:100E6E000F1B900771E0B43C028003020F05C29C79
:100E7E0012053F12013590006CE09000E0F09000FA
:100E8E006DE0900097F090006EE0900098F0A21A3E
:100E9E004032755001E550D394075026E550900727
:100EAE00B1F8E4F0E8A3F074AA90003DF0123223FA
:100EBE007464F5097508001231F77850740126F63E
:100ECE0050D38030755008E550D3940E5026E5501F
:100EDE009007B1F8E4F0E8A3F074AA90003DF01288
:100EEE0032237464F5097508001231F778507401D5
:100EFE0026F650D31235F774C89007B1F8E4F0E82F
:100F0E00A3F0D29C7547007546007599FBE547B472
:100F1E0002028003020FC5E5324531700685992E17
:100F2E00752D00AE31AF3274016F4E701BAC2DAD0E
:100F3E002EAA2FAB30ED2BFBEC3AFA8A068B0790DC
:100F4E0000711252E8E599F0783112531EAE31AFAE
:100F5E003274026F4E7060AC2DAD2E740D6D4C70F0
:100F6E002C74639007B1F8E4F0E8A3F074AB900032
:100F7E003DF090007EE090005AF012355C90003DFE
:100F8E00E4F074C89007B1F8E4F0E8A3F0E548B4D3
:100F9E00E619AE2DAF2E74566F4E600C74486F4E20
:100FAE00600674666F4E700312053F120135854858
:100FBE0099754700754600E547B4033FAE31AF3231
:100FCE009000711252E8E599F0783112531EAE314D
:100FDE00AF32AC2FAD308F028E038C068D07905042
:100FEE0073125282E493F9740193FEEAD39EEB9945
:100FFE004009854899754700754600E547B40402D7
:10100E008003021168AE31AF329000711252E8E5E2
:10101E0099F0783112531EAE31AF32EFB40006EEB6
:10102E00B40102800302116812053F900053E0756F
:10103E00F002A4FFAEF08F50EF9000711252F3EF5A
:10104E00FCE0FDEC9000741252F3EDFCE0FDEC2D93
:10105E00FC900053E0B5040280030211590FEF908B
:10106E0000711252F3E550FFE0FCEF900075125242
:10107E00F3ECFFE0FCEFC39CFF900053E0B50702DA
:10108E008003021159E5509000731252F3E550FFA0
:10109E00E0FCEF9000761252F3ECFFE0FCEF2CFF39
:1010AE00900053E0B507028003021159E5509000FD
:1010BE00771252F3FFE0FCEF900053E0F4042C9013
:1010CE00005AF0E5509000781252F3FFE0FCEF90DA
:1010DE000053E0F4042C90005BF0E5509000791280
:1010EE0052F3FFE0FCEF900053E0F4042C90005C10
:1010FE00F0E55090007A1252F3FFE0FCEF900053AF
:10110E00E0F4042C9007B1F8E4F0E8A3F074AB908F
:10111E00003DF012355C7464F5097508001231F764
:10112E009007B11252CF12355C7464F50975080040
:10113E001231F79007B11252CF12355C7599F974CE
:10114E0064F5097508001231F780FE7599FF746415
:10115E00F5097508001231F780FEE5466006A29982
:10116E00B3B340030212E8C299E546B4011FAE3193
:10117E00AF329000491252E8E0F599783112531EC1
:10118E00AE31AF3274116F4E7003754600E546B442
:10119E000203854A99E546B4031DAE31AF32900085
:1011AE00711252E8E0F599EFB40107EEB40703753A
:1011BE004600783112531EE546B404028003021233
:1011CE00AAE53245317003852699AE31AF327401EE
:1011DE006F4E7003853899AE31AF3274026F4E7018
:1011EE0003853A99AE31AF3274036F4E7003853E6C
:1011FE0099AE31AF3274046F4E7003854099AE31A3
:10120E00AF3274056F4E7003854199AE31AF3274B3
:10121E00066F4E7003854299AE31AF3274076F4E32
:10122E007003854399AE31AF3274086F4E700690DD
:10123E00001BE0F599AE31AF3274096F4E7017A2F4
:10124E0021B340077599FAC221800B900045E0F555
:10125E0099900045E4F0AE31AF32740A6F4E7003D0
:10126E00854499AE31AF32740B6F4E7003853F9942
:10127E00AE31AF32740C6F4E7003854599AE31AFFF
:10128E0032740D6F4E70037599FC783112531EAE89
:10129E0031AF32740E6F4E7003754600E546B405DD
:1012AE003990004BE0D394044010AE31AF32904DE4
:1012BE00EB1252E8E493F599800EAE31AF32904EB8
:1012CE00CF1252E8E493F599AE31AF3274E36F4E1C
:1012DE007003754600783112531EE54764016005B0
:1012EE00E547B40403020D5AC28E7E107F00E53D21
:1012FE001252C1E58D75F010A4FDACF0EF2DFDEE90
:10130E003CFCE58B75F01084FF7E00ED2FFFEC3E6C
:10131E00FE8E278F28D28E90009EE0605690001C85
:10132E001252CF90001CE0FCA3E0FD90001EE0FAEC
:10133E00A3E0FBEDB5033CECB50238B219A208B33D
:10134E004013A219B34008E5B54404F5B58006E58F
:10135E00B554FBF5B590001EE0FEA3E0FF90002013
:10136E00E0FCA3E0FDEF2DFDEE3CFC90001EECF04A
:10137E00A3EDF09000ABE060099000ABE0C39403E6
:10138E00400302143E124B31A208B350099000687C
:10139E00E0C3942840028006900095E0F56BE56B63
:1013AE0075F005A4FFAEF09007B3EEF0A3EFF0904A
:1013BE000082E0C3953A4007E538C395395007904F
:1013CE0007B3E4F0A3F0AE58AF599007B3E0FCA317
:1013DE00E0FDEFD39DEE9C4028E5B5547FF5B5902A
:1013EE0000ABE0B402119000D7E0640160099000F8
:1013FE00C9E0C3940240028006E5B54440F5B580CD
:10140E002F900068E0C3943C5026E5B54480F5B5B6
:10141E009000ABE0B402119000D7E0640160099037
:10142E0000C9E0C3940240028006E5B554BFF5B58D
:10143E009000ABE0B40324124C4CAE58AF59900759
:10144E00B3E0FCA3E0FDEFD39DEE9C4008E5B54470
:10145E0080F5B58006E5B5547FF5B5900086E06061
:10146E0009A2B3300A01B3B340028028A2B3300AF6
:10147E0001B34020A2B3300C01B3400B900070E0DA
:10148E0004F0A20CB3920AA20CB330B301B3400421
:10149E00A20C920AA2B6300901B35003021A3CA262
:1014AE00B6300901B35003021A3CA2B6300B01B399
:1014BE005003021972754A0090009EE07013A20B41
:1014CE00B34008E5B554FBF5B58006E5B54404F523
:1014DE00B50537A20DB3B35013AE27AF2890000C4D
:1014EE00E0FCA3E0FDEDC39FEC9E400302162090AE
:1014FE000070E0B40104C21C8019900070E0B402C8
:10150E0004D21C800EB21C900070E0700674049021
:10151E000045F0900070E4F0E549B40330E537B4CF
:10152E002305754901801FA222B3401AE537C394E3
:10153E002350069000457401F0E537D394234006FE
:10154E007402900045F0753701D222805CE549B4F3
:10155E000206754901753723E537B4230575370142
:10156E008047900045E07032E537C39423500690D3
:10157E0000457401F0E537D39423400674029000C1
:10158E0045F0E537C394235002D21FE537D3942399
:10159E004002D21FC296C295C2A09000BBE0B40218
:1015AE000512053F8003753701AE29AF2AAC27AD72
:1015BE0028EF2DFDEE3CFC74028C068D071252B303
:1015CE008E298F2A90009EE0603F90001CE0FCA3C5
:1015DE00E0FD90009EE0FF1252A374018C068D0771
:1015EE001252B3900020EEF0A3EFF0900020E0F83E
:1015FE00A3E090001EC8F0A3C8F090001CE4F0A376
:10160E00F0C219E5B554FBF5B5A21FB34002C21FD7
:10161E00802BAE29AF2AAC27AD28EF2DFDEE3CFC7A
:10162E0074018C068D071252B38E298F2AAC27AD0A
:10163E0028EDD39488EC9413400312053FE537B49C
:10164E0023127403900045F0D21F9000BBE0B40249
:10165E000312053FAE2BAF2CAC27AD28EF2DFDEEC0
:10166E003CFC8C2B8D2CAE27AF28EFD39DEE9C40EF
:10167E0011900014E0FAA3E0FBEBC394E8EA9403A4
:10168E00400280069000141252CF900010E0FEA38C
:10169E00E0FFAC27AD28EF2DFDEE3CFC900010ECEA
:1016AE00F0A3EDF09000BBE0B40218AE27AF2874A3
:1016BE00051252C174011252B390000CEEF0A3EF5A
:1016CE00F08011AE27AF2874021252C190000CEEBA
:1016DE00F0A3EFF0C28E758D00758B00753D007511
:1016EE002801752700D28EE537240875F00984AFDE
:1016FE00F07E00EF4E7075900010E0F8A3E09000C1
:10170E000EC8F0A3C8F090000EE0FEA3E0FFEF4E6F
:10171E00600B7C807D0E1251A18E258F26900010BD
:10172E00E4F0A3F0AE25AF267428BE00039F501040
:10173E00E53C2FFF50010E74011252B38E258F26F9
:10174E0085263C9000C2E0A825B8000DD395264012
:10175E0008E526900042F080099000C2E014900047
:10176E0042F0E5496006752600752500E537640BE5
:10177E006005E537B41D099000ABE06003124839EF
:10178E009000B0E0B4011490003EE0653760079021
:10179E00003FE0B53703754B00801E90003EE065BC
:1017AE0037601390003EE0240C6537600990003ED0
:1017BE00E02418B53703754B00A20EB35006A20DE8
:1017CE00B3B340030218C7900077E0B4015AE54066
:1017DE0075F00584FF7E009005711252E8E0F53435
:1017EE00753300AE33AF34900075E01252C174649D
:1017FE008E048F05FF1252A374C18C068D071252F0
:10180E00C18E358F36900012E0FEA3E0FFAC33ADF3
:10181E003412000374648E048F05FF1252A39000DD
:10182E0012ECF0A3EDF0800F900075E075F0C1A4FE
:10183E00FFAEF08E358F36E53AC394CC500690004D
:10184E0075E07002807175A71085F95085FA517E8A
:10185E00017F00E5511252C1E5502FFF50010E8E4F
:10186E00338F34AC35AD36EF2DFDEE3CFC8C358D23
:10187E0036D293D294D291E536F5FBE535F5FCE5FB
:10188E0036F5E9E535F5EAE536F5EBE535F5EC90B7
:10189E0000B9E0B4031ED292D287D290E536F5EDB0
:1018AE00E535F5EEE536F5FDE535F5FEE536F5CE35
:1018BE00E535F5CF75A700D20EE549B40106E5373B
:1018CE00640B6002800F754C019000487401F0E5C6
:1018DE00B54401F5B5E549600302196D9000BEE00F
:1018EE00600D9000C5E0A825B80006952640028040
:1018FE003A9000BEE0B4021F900034E06537600FEE
:10190E00900035E065376007900036E0B537037517
:10191E004C03754500800CC20075450090001AE41A
:10192E00F0A3F07409900045F08034900034E0B5D7
:10193E00370B754C019000487401F08022900035F1
:10194E00E0B5370B754C017402900048F080109092
:10195E000036E0B53709754C017403900048F0A2CB
:10196E000BB39209A20BB330B601B35003021A3C6B
:10197E00754A0190009EE07013A20BB34008E5B5C6
:10198E004404F5B58006E5B554FBF5B5A20B9209F6
:10199E00E537D3944A4014D20DE537D3946D400BFE
:1019AE007403900045F0D21F7537469000C6E0B420
:1019BE000107E543C394144002800312053F7428C7
:1019CE00900068F0A204300501B35017A204B34092
:1019DE0008E5B54408F5B58006E5B554F7F5B5A2AA
:1019EE00049205E543C394415009740E900045F0EE
:1019FE0012053F90004FE0FE90004BE004C39E4066
:101A0E000990004BE0D39406400974FB900045F01A
:101A1E0012053F900054E06015900054E0FE9000D7
:101A2E004EE06E600974FE900045F012053FA21F55
:101A3E00B34006C296C295C2A0A210B3B35008908E
:101A4E000037E065376003021B45A202B35006A2C1
:101A5E0000B3B34003021B3F75A71085F95085FAFA
:101A6E00517E017F00E5511252C1E5502FFF50010A
:101A7E000E8E338F34900018E0FCA3E0FDEF2DFDA9
:101A8E00EE3CFC8C358D369000B9E0B4035EA208B6
:101A9E00B34030A21CB3400CE536F5FBE535F5FC42
:101AAE00D293800AE536F5EDE535F5EED292A20336
:101ABE00B34008E5B54440F5B58006E5B554BFF52D
:101ACE00B58027E536F5FBE535F5FCE536F5EDE5B4
:101ADE0035F5EED293D292A203B34008E5B5444059
:101AEE00F5B58006E5B554BFF5B580429000D7E058
:101AFE00C394025013E536F5FBE535F5FCD293A2FF
:101B0E0003B34002D2928026E536F5FBE535F5FCAF
:101B1E00D293AE33AF34AC56AD57EF2DFDEE3CFC49
:101B2E008C358D36E536F5EDE535F5EED29275A7A9
:101B3E0000C210D211D212A211B3B35008900038C5
:101B4E00E065376003021C43A202B35006A200B345
:101B5E00B34003021C3D75A71085F95085FA517EDE
:101B6E00017F00E5511252C1E5502FFF50010E8E3C
:101B7E00338F34900018E0FCA3E0FDEF2DFDEE3C1A
:101B8E00FC8C358D369000B9E0B4035EA208B340EC
:101B9E0030A21CB3400CE536F5E9E535F5EAD294F2
:101BAE00800AE536F5FDE535F5FED287A203B34092
:101BBE0008E5B54440F5B58006E5B554BFF5B580EA
:101BCE0027E536F5E9E535F5EAE536F5FDE535F5D2
:101BDE00FED294D287A203B34008E5B54440F5B5D2
:101BEE008006E5B554BFF5B580429000D7E0C394AA
:101BFE00025013E536F5E9E535F5EAD294A203B3C2
:101C0E004002D2878026E536F5E9E535F5EAD2942D
:101C1E00AE33AF34AC56AD57EF2DFDEE3CFC8C35EC
:101C2E008D36E536F5FDE535F5FED28775A700D282
:101C3E0010C211D212A212B3B35008900039E0654F
:101C4E00376003021D41A202B35006A200B3B34097
:101C5E0003021D3B75A71085F95085FA517E017F51
:101C6E0000E5511252C1E5502FFF50010E8E338FF9
:101C7E0034900018E0FCA3E0FDEF2DFDEE3CFC8C53
:101C8E00358D369000B9E0B4035EA208B34030A2A1
:101C9E001CB3400CE536F5EBE535F5ECD291800A38
:101CAE00E536F5CEE535F5CFD290A203B34008E583
:101CBE00B54440F5B58006E5B554BFF5B58027E5CA
:101CCE0036F5EBE535F5ECE536F5CEE535F5CFD267
:101CDE0091D290A203B34008E5B54440F5B5800615
:101CEE00E5B554BFF5B580429000D7E0C3940250DD
:101CFE0013E536F5EBE535F5ECD291A203B34002D0
:101D0E00D2908026E536F5EBE535F5ECD291AE3383
:101D1E00AF34AC56AD57EF2DFDEE3CFC8C358D3609
:101D2E00E536F5CEE535F5CFD29075A700D210D2B7
:101D3E0011C212E54CB40818124168A210B3500536
:101D4E00A211B340028006D210D211D212754C1ECF
:101D5E00E54CB40706123F20754C08E54CB4063D21
:101D6E00900012E0FEA3E0FFEF4E6006A208B3B3B0
:101D7E0040028023AE52AF53900012E0FCA3E0FD70
:101D8E00EF2DFDEE3CFC8C528D53E537D3940C5069
:101D9E0006900012120039123CF2754C07E54CB455
:101DAE000506123B52754C06E54CB404329000AC5D
:101DBE00E09031D9F82828731237E680121237E6F0
:0F1DCE00800D1239948008123A468003123A466B
:0F31D900021DC6021DCB021DD0021DD5021DDA3C
:101DDD0090008EE060051249228002C204754C0508
:101DED00E54CB403028003021ED7900091E060051C
:101DFD00124A2F8002C2069000ACE0D39402403FFD
:101E0D00900080E02403A825B80004952650099081
:101E1D000082E0D3953A50028008D20274089000F7
:101E2D0045F0900080E0A825B80005D39526500B0D
:101E3D00900082E02403C3953A5002C2028039908B
:101E4D000080E02403A825B8000495265007E53846
:101E5D00C3953940028008D2027408900045F09075
:101E6D000080E0A825B80005D395265009E5392452
:101E7D000FC395385002C2029000C6E07007E543CB
:101E8D00C3941440028002D202A2024005754C0494
:101E9D00800A754C1E90001AE4F0A3F0A208B3401E
:101EAD0029E54075F00584FF7E009005711252E81A
:101EBD00E0C39469500512486E800F9007ABE0F8AF
:101ECD00A3E09007A9C8F0A3C8F0E54CB40A0280BE
:101EDD0003021F9990002AE0C394465008C29674DD
:101EED004690002AF090003AE0B4011DE55A240A0C
:101EFD00F55A9007ADE0FEA3E0FF740A2FFF5001E5
:101F0D000E9007ADEEF0A3EFF090003AE0B4021D95
:101F1D00E55A2414F55A9007ADE0FEA3E0FF7414C2
:101F2D002FFF50010E9007ADEEF0A3EFF0855A3460
:101F3D00753300900034E0F55012009EE5369000A8
:101F4D002AF0900006E533F0A3E534F0E55090005B
:101F5D002BF0C2149007ADE0F533A3E0F5349000FB
:101F6D0034E0F55012009EE536900028F090000008
:101F7D00E533F0A3E534F0E550900029F0C213E508
:101F8D0049B40105754C0B8003754C03900028E096
:101F9D00B53702800302203BA2134072900000E08F
:101FAD00FEA3E0FFEF4E6021AE29AF2A900000E0C6
:101FBD00FCA3E0FD120003740A8E048F05FF12527C
:101FCD00A3900000ECF0A3EDF0900029E0601A90D2
:101FDD000000E0FEA3E0FFAC29AD2AEF2DFDEE3CA5
:101FED00FC900000ECF0A3EDF0900029E0D39401FB
:101FFD00401A900000E0FEA3E0FFAC29AD2AEF2DC2
:10200D00FDEE3CFC900000ECF0A3EDF0D213AE27FA
:10201D00AF28900000E0FCA3E0FDEFC39DEE9C40D7
:10202D000D12060ED296C21374C8900028F0A2139A
:10203D00B3B35007900028E0B53702800D12060E9D
:10204D00D29674C8900028F0C21390002AE0B537DC
:10205D000280030220F6A2144072900006E0FEA357
:10206D00E0FFEF4E6021AE29AF2A900006E0FCA301
:10207D00E0FD120003740A8E048F05FF1252A39027
:10208D000006ECF0A3EDF090002BE0601A90000636
:10209D00E0FEA3E0FFAC29AD2AEF2DFDEE3CFC9058
:1020AD000006ECF0A3EDF090002BE0D39401401A64
:1020BD00900006E0FEA3E0FFAC29AD2AEF2DFDEE6A
:1020CD003CFC900006ECF0A3EDF0D214AE27AF2847
:1020DD00900006E0FCA3E0FDEFC39DEE9C400AC21C
:1020ED0096744690002AF0C214A214B3B350079010
:1020FD00002AE0B53702800AC296744690002AF095
:10210D00C214E54CB40B0280030221DC90002EE0DA
:10211D00C3944650139000C7E0B40104C2968002E8
:10212D00C295744690002EF090003BE0B4011DE581
:10213D005A240AF55A9007ADE0FEA3E0FF740A2F6A
:10214D00FF50010E9007ADEEF0A3EFF090003BE0D5
:10215D00B4021DE55A2414F55A9007ADE0FEA3E034
:10216D00FF74142FFF50010E9007ADEEF0A3EFF0AA
:10217D00855A34753300900035E0F55012009EE518
:10218D003690002EF0900008E533F0A3E534F0E52D
:10219D005090002FF0C2169007ADE0F533A3E0F597
:1021AD0034900035E0F55012009EE53690002CF08D
:1021BD00900002E533F0A3E534F0E55090002DF0EA
:1021CD00C215E549B40105754C0C8003754C03909F
:1021DD00002CE0B537028003022289A215407290CF
:1021ED000002E0FEA3E0FFEF4E6021AE29AF2A9082
:1021FD000002E0FCA3E0FD120003740A8E048F05BB
:10220D00FF1252A3900002ECF0A3EDF090002DE030
:10221D00601A900002E0FEA3E0FFAC29AD2AEF2D7D
:10222D00FDEE3CFC900002ECF0A3EDF090002DE0F3
:10223D00D39401401A900002E0FEA3E0FFAC29AD5B
:10224D002AEF2DFDEE3CFC900002ECF0A3EDF0D258
:10225D0015AE27AF28900002E0FCA3E0FDEFC39D73
:10226D00EE9C401812060E9000C7E0B40104D29601
:10227D008002D295C21574C890002CF0A215B3B38C
:10228D00500790002CE0B53702801812060E900012
:10229D00C7E0B40104D2968002D29574C890002C88
:1022AD00F0C21590002EE0B53702800302235AA22A
:1022BD00164072900008E0FEA3E0FFEF4E6021AEE5
:1022CD0029AF2A900008E0FCA3E0FD120003740A78
:1022DD008E048F05FF1252A3900008ECF0A3EDF0D1
:1022ED0090002FE0601A900008E0FEA3E0FFAC29FB
:1022FD00AD2AEF2DFDEE3CFC900008ECF0A3EDF0C7
:10230D0090002FE0D39401401A900008E0FEA3E066
:10231D00FFAC29AD2AEF2DFDEE3CFC900008ECF052
:10232D00A3EDF0D216AE27AF28900008E0FCA3E095
:10233D00FDEFC39DEE9C40159000C7E0B40104C2B3
:10234D00968002C295744690002EF0C216A216B366
:10235D00B3500790002EE0B5370280159000C7E00E
:10236D00B40104C2968002C295744690002EF0C24C
:10237D0016E54CB40C028003022449900032E0C3F0
:10238D00944650139000C7E0B40104C2968002C277
:10239D00A07446900032F090003CE0B4011DE55A67
:1023AD00240AF55A9007ADE0FEA3E0FF740A2FFF53
:1023BD0050010E9007ADEEF0A3EFF090003CE0B4AD
:1023CD00021DE55A2414F55A9007ADE0FEA3E0FF77
:1023DD0074142FFF50010E9007ADEEF0A3EFF085B2
:1023ED005A34753300900036E0F55012009EE536F4
:1023FD00900032F090000AE533F0A3E534F0E5509B
:10240D00900033F0C2189007ADE0F533A3E0F5343A
:10241D00900036E0F55012009EE536900030F090B9
:10242D000004E533F0A3E534F0E550900031F0C23F
:10243D0017E549B40103754900754C03900030E070
:10244D00B5370280030224F6A2174072900004E013
:10245D00FEA3E0FFEF4E6021AE29AF2A900004E00D
:10246D00FCA3E0FD120003740A8E048F05FF1252C7
:10247D00A3900004ECF0A3EDF0900031E0601A9011
:10248D000004E0FEA3E0FFAC29AD2AEF2DFDEE3CEC
:10249D00FC900004ECF0A3EDF0900031E0D394013A
:1024AD00401A900004E0FEA3E0FFAC29AD2AEF2D09
:1024BD00FDEE3CFC900004ECF0A3EDF0D217AE273E
:1024CD00AF28900004E0FCA3E0FDEFC39DEE9C401F
:1024DD001812060E9000C7E0B40104D2968002D205
:1024ED00A0C21774C8900030F0A217B3B350079074
:1024FD000030E0B53702801812060E9000C7E0B428
:10250D000104D2968002D2A074C8900030F0C21798
:10251D00900032E0B5370280030225C7A218407241
:10252D0090000AE0FEA3E0FFEF4E6021AE29AF2A36
:10253D0090000AE0FCA3E0FD120003740A8E048FE4
:10254D0005FF1252A390000AECF0A3EDF0900033BA
:10255D00E0601A90000AE0FEA3E0FFAC29AD2AEF7F
:10256D002DFDEE3CFC90000AECF0A3EDF090003355
:10257D00E0D39401401A90000AE0FEA3E0FFAC29DD
:10258D00AD2AEF2DFDEE3CFC90000AECF0A3EDF032
:10259D00D218AE27AF2890000AE0FCA3E0FDEFC3F0
:1025AD009DEE9C40159000C7E0B40104C2968002D8
:1025BD00C2A07446900032F0C218A218B3B35007EF
:1025CD00900032E0B5370280159000C7E0B40104E9
:1025DD00C2968002C2A07446900032F0C218E54C3B
:1025ED00B40202800302269B1245D11246E89007E1
:1025FD00A9E0FEA3E0FF740A1252C190000EE0FCA8
:10260D00A3E0FD74098F02FF1252A38D078C038E78
:10261D00048A058B061251A19007ADEEF0A3EFF0E1
:10262D009000C7E0B401087450BE00059F400280C1
:10263D000D74509007ADF8E4F0E8A3F0801B9007FF
:10264D00ADE0FEA3E0FF74F0BE00039F500B74F0ED
:10265D009007ADF8E4F0E8A3F09007ADE0FEA3E03D
:10266D00FFE55A2FFF50010E9007ADEEF0A3EFF0EE
:10267D00900048E0B40103754C0A900048E0B402A4
:10268D0003754C0B900048E0B40303754C0CE54CFE
:10269D00B401259000DEE09031E8F828287312434C
:1026AD006F801212436F800D1243F980081244A5FA
:0526BD0080031244A59A
:0F31E8000226AB0226B00226B50226BA0226BF87
:1026C200754C029000C9E0B4020280030227E9902F
:1026D200006BE0D3953F506490006BE0F404253F1B
:1026E200FE9000CCE08E00F5F0E884FF7E008F5073
:1026F200EFC39410500CEF8550F0A4FDACF08D5058
:1027020080037550FF90006BE0D39550400B900012
:102712006BE0C39550F54D8003754D009000E7E0E6
:10272200D3954D40069000E7E0F54D9000E8E0C3F8
:10273200954D50069000E8E0F54D807190006BE0F9
:10274200C3953FFE9000CCE08E00F5F0E884FF7E5A
:10275200008F50EFC39410500CEF8550F0A4FDACE5
:10276200F08D5080037550FF855034753300900012
:102772006BE02534FFAE3350010E8E338F3474FF7D
:10278200BE0009D39F400585344D8003754DFF90EF
:1027920000E7E0D3954D40069000E7E0F54D90004C
:1027A200E8E0C3954D50069000E8E0F54DA208B36D
:1027B200B350099000D4E0D3954E5002800E7407B6
:1027C200900045F0E5B554BFF5B5801B75A710E53F
:1027D200CDC3954D4008E5B554BFF5B58006E5B5C6
:1027E2004440F5B575A700A206B3402575A710A20F
:1027F20008B3B35007E5CDC394BF40028008E5B5E6
:102802004420F5B58006E5B554DFF5B575A700801F
:102812002375A710A208B3B35007E5CDC394404077
:10282200028008E5B54420F5B58006E5B554DFF52C
:10283200B575A700E54BC394094003022F71A2EDC1
:10284200B35003022F71C2EDE54B60030229E590FC
:10285200007AE070030229D49000B0E0B401028053
:102862000302293490003EE0B53702800302293189
:102872007E017F00E5BE1252C1E5BD2FFF50010E61
:102882008E338F3490007AE0B4011874101252C162
:1028920090006FE08E048F05FF1252A3ED9000406E
:1028A200F0802CAE33AF3474101252C190006FE03E
:1028B2008E048F05FF1252A3900040E02DFD5001BF
:1028C2000C74018C068D071252B3EF900040F0E5B4
:1028D2004460089000D6E06402600280219000D833
:1028E200E0B4011A900040E075F0E7A4FFAEF0E515
:1028F200448E048F05FF1252A3ED900040F0900029
:1029020040E0FE900041E0D39E4004D21D8002B21E
:102912001D900040E0900041F09000ACE064016046
:1029220006A21DB3B340028006900040E0F53802D3
:1029320029D2D21D7E017F00E5BE1252C1E5BD2F14
:10294200FF50010E8E338F3490007AE0B401187478
:10295200101252C190006FE08E048F05FF1252A335
:10296200ED900040F0802CAE33AF3474101252C19F
:1029720090006FE08E048F05FF1252A3900040E09A
:102982002DFD50010C74018C068D071252B3EF908D
:102992000040F0E54460089000D6E06402600280E6
:1029A200219000D8E0B4011A900040E075F0E7A44D
:1029B200FFAEF0E5448E048F05FF1252A3ED9000A6
:1029C20040F09000ACE064016006900040E0F53811
:1029D2008003753800900076E07005754B01800326
:1029E20075BB18E54BB401028003022B8790007679
:1029F200E07003022B767E017F00E5BE1252C1E534
:102A0200BD2FFF50010E8E338F349000BCE0B40115
:102A12000F7E0F7FFFAC33AD341253168E338F34DB
:102A22009000E1E0B40245AE33AF34900024E0FC04
:102A3200A3E0FDEDD39FEC9E400A900024E533F025
:102A4200A3E534F0AE33AF34900026E0FCA3E0FD02
:102A5200EFD39DEE9C400A900026E533F0A3E534C7
:102A6200F0AE33AF3474041252B38F3A9000E1E007
:102A7200704CAE33AF34900024E0FCA3E0FDEFD302
:102A82009DEE9C40091253168E338F3480067534A6
:102A920000753300AE33AF3474101252C190006C23
:102AA200E08E048F05FF1252A38C338D347400D351
:102AB2009D74019C400585343A8003753AFF90006D
:102AC200ACE0B401028003022B74A208B3B3500E2F
:102AD200900080E0A825B80005D395265003022B6C
:102AE20069900081E075F019A4FFAEF09000C4E097
:102AF2008E048F05FF1252A39000BDE0853AF0A428
:102B0200FFAEF074648D028C038E048F05FF1252A7
:102B1200A3EA2DFDEB3CFC8C338D34E544600F9031
:102B220000D6E0B402089000D8E064016002801789
:102B3200AE33AF3474E71252C1E5448E048F05FF01
:102B42001252A38C338D34900040E0A833B8000AAF
:102B5200D395344005853438800BA21DB3400690CE
:102B62000040E0F538800BA21DB34006900040E023
:102B7200F5388003753A00900079E07005754B02D4
:102B8200800375BB19E54BB402028003022C42900C
:102B92000079E07003022C31E537D3940C40030234
:102BA2002C2F900022E0FEA3E0FFE53E12530E9090
:102BB2000022EEF0A3EFF07E017F00E5BE1252C1CB
:102BC200E5BD2FFF50010E8E338F349000E6E0708A
:102BD20013740A1252C174518E048F05FF1252A34C
:102BE2008D3E8019AE33AF34740A1252C18F048EF7
:102BF200057E017F95CDCCCD1251A18F3EE53ED30E
:102C020094644003753E64900022E0FEA3E0FFE579
:102C12003E2FFF50010E900022EEF0A3EFF0900045
:102C22007DE0048E048F05FF1252A38D3E80037552
:102C32003E329000C9E07005754B03800375BB13EB
:102C4200E54BB4035E9000C9E060477E017F00E57A
:102C5200BE1252C1E5BD2FFF50010E8E338F347468
:102C6200041252B38F3F9000CBE0853FF0A4FDAC3D
:102C7200F07464FF1252A38D3F9000CAE0853FF0CA
:102C8200A4FFAEF074FF8E048F05FF1252A38D4E87
:102C92008003753F00900077E07005754B04800358
:102CA20075BB17E54BB404028003022D43900077F5
:102CB200E0B4017C7E017F00E5BE1252C1E5BD2F6A
:102CC200FF50010E74041252B38E338F34900043BE
:102CD200E06012900043E0149050AF93A833B80024
:102CE20006953440028006900043E014F0900043C1
:102CF200E0C394775013900043E0049050AF93A840
:102D020033B80005D3953450028006900043E004A6
:102D1200F0900043E0FE90009DE08E0088F0A4FF5A
:102D2200AEF074648E048F05FF1252A38D408003AF
:102D3200754000900078E07005754B05800375BB07
:102D420016E54BB405028003022DD6900078E0B45C
:102D5200017C7E017F00E5BE1252C1E5BD2FFF500E
:102D6200010E74041252B38E338F34900044E0602B
:102D720012900044E01490512893A833B8000695AD
:102D82003440028006900044E014F0900044E0C316
:102D920094775013900044E00490512893A833B8DC
:102DA2000005D3953450028006900044E004F09070
:102DB2000044E0FE9000A3E08E0088F0A4FFAEF095
:102DC20074648E048F05FF1252A38D4180037541F6
:102DD2000075BB1FE54BB406337E017F00E5BE12D2
:102DE20052C1E5BD2FFF50010E8E338F347409128C
:102DF20052C174E68E048F05FF1252A38D439000D8
:102E02007FE07005754B07800375BB15E54BB40772
:102E1200028003022F1890007FE07003022F077ECA
:102E2200017F00E5BE1252C1E5BD2FFF50010E8E9B
:102E3200338F3474041252B38F4290007FE0B40196
:102E4200159000D3E08542F0A4FFAEF07407125251
:102E5200B3EF9007B6F090007FE0B402159000D374
:102E6200E08542F0A4FFAEF074071252B3EF900770
:102E7200B5F090007FE0B403028003022F059000BA
:102E8200C0E0701CE542C3940A5002D201E542D36D
:102E920094644002C20190009FE090006AF0806357
:102EA20090009FE070349000D3E08542F0A4FFAE22
:102EB200F074FF8E048F05FF1252A3ED90006AF0AA
:102EC200AE25AF26741EBE0006D39F4002D201E596
:102ED2003AD394E54002C2018029E542C3940A50E4
:102EE2000DAE25AF26741EBE0004D39F5002800291
:102EF200D201E53AD394E54002C20190009FE090EE
:102F0200006AF080037542009000D6E07005754BB0
:102F120008800375BB14E54BB408509000D6E060FE
:102F2200397E017F00E5BE1252C1E5BD2FFF50017F
:102F32000E8E338F34EFD39421EE940E40057544F8
:102F4200FF8015AE33AF3474101252C174E38E0495
:102F52008F05FF1252A38D44800375440090007ABE
:102F6200E0600575BB1A800375BB18054BD2ECAE49
:102F720027AF287498C39F743A9E400C900069E072
:102F8200C3943C40030231D6C20D7537469000BB54
:102F9200E070057549028003754903C293C294C269
:102FA20091C292C287C290E5B554EFF5B5E5B5542A
:102FB200DFF5B5C296C295C2A0C297C2A2C2A1E570
:102FC200B554BFF5B5E5B5547FF5B5A21EB34008BB
:102FD200E5B54404F5B58006E5B554FBF5B5A20F99
:102FE200B3500EE53AD394334007E53AC394CC404C
:102FF20003023093E5B54401F5B57428900068F0FA
:10300200900075E075F064A4FFAEF08E358F3674D3
:1030120002BE000AD39F400675360275350075A7B9
:103022001085F95085FA517E017F00E5511252C197
:10303200E5502FFF50010E8E338F34AC35AD36EF95
:103042002DFDEE3CFC8C358D36D293D294D291E597
:1030520036F5FBE535F5FCE536F5E9E535F5EAE566
:1030620036F5EBE535F5EC9000B9E0B4031ED292EB
:10307200D287D290E536F5EDE535F5EEE536F5FD8C
:10308200E535F5FEE536F5CEE535F5CF75A700D287
:103092000FE53AC3941A5002C20F90000C74FFF06D
:1030A200A374DCF090009CE0900012F8E4F0E8A336
:1030B200F0C213C215C21774C8900028F074C890E9
:1030C200002CF074C8900030F0C210C211C2127508
:1030D2002600752500753C00C208756C0090001A28
:1030E200E4F0A3F0754C1E9007ABE0FEA3E0FF7482
:1030F200031252C174011252B39007A9EEF0A3EF6A
:10310200F090008EE060051249228002C204900015
:1031120091E06005124A2F8002C206A20430050126
:10312200B35017A204B34008E5B54408F5B58006CC
:10313200E5B554F7F5B5A2049205C203752C0075E6
:103142002B00900014E4F0A3F090007DE075F032C3
:10315200A4FFAEF0900022EEF0A3EFF0900010E496
:10316200F0A3F0C222900069E0C3943C5010E54BFA
:10317200B40909900069E004F0754B00803BE54B0F
:10318200B40903754B00752800752700758D00750D
:103192008B00753D00900068E0C3943C500890009D
:1031A20068E004F08006743C900068F0900068E0EB
:1031B200B43C06E5B554FEF5B5900069E0D3940140
:1031C2004007E543C3944140028009740E900045D4
:0731D200F012053F020D5A47
:105037000000010001400160018001A001C001E002
:1050470002000300039603B603D603F40400050029
:1050570005180530054805600578059005A805C0C1
:10506700060006140628063C066E068C00FF013F64
:10507700015F017F019F01BF01DF01FF02FF039570
:1050870003B503D503F303FF04FF0517052F0547F2
:10509700055F0577058F05A705BF05FF06130627DB
:1050A700063B066F068B06A9DAD8D7D5D4D2D0CF60
:1050B700CDCBC9C7C6C4C2C0BEBCBAB8B5B3B1AF01
:1050C700ADABA8A6A4A2A09D9B99969492908D8B18
:1050D70089878482807E7C79777573716F6D6B6940
:1050E700676563615F5D5B5957565452504F4D4B2F
:1050F7004A4847454442413F3E3C3B3A39373635BB
:10510700343231302F2E2D2C2B2A292827262525DE
:105117002423222121201F1E1E1D1C1C1B1A1A19A5
:1051270019EEECEBEAE9E8E7E5E4E3E1E0DEDDDBF5
:10513700D9D8D6D4D2D0CECCCAC8C6C3C1BFBCBAC0
:10514700B7B5B2B0ADABA8A5A3A09D9B989592901B
:105157008D8A8785827F7D7A7775726F6D6A6865BC
:1051670063615E5C5A575553514F4D4B4947454311
:1051770042403E3C3B393836353332312F2E2D2BCA
:105187002A292827262524232221201F1E1D1D1CEE
:0A5197001B1A1A191818171616151E
:1031F700750B00750A00AE0AAF0BAC08AD09EDC33D
:103207009FEC9E401674FF12529375CF01780B7492
:103217000126F6500418E436F650DB2290003DE014
:10322700B4AA1C900771E0B43C159007B1E0FEA367
:10323700E0FFEF4E6009741EBE0004D39F500302E7
:10324700335175360075350075F8099007B1E0FE02
:10325700A3E0FF74076F4E6006740E6F4E7006741E
:103267003A900771F09007B1E0FEA3E0FF7408BE43
:10327700001ED39F401A7E017F089007B1E0FCA390
:10328700E0FD1DBDFF011C1200038E338F34801F2C
:103297009007B1E0FEA3E0FF740812530E8F048E6F
:1032A700057E017F08CDCCCD1200038E338F34AE5F
:1032B70035AF36740CD39F74019E500302334CA272
:1032C700F9B3407EE5364535700375A382AE35AF59
:1032D7003674016F4E700375A300AE35AF367402B6
:1032E7006F4E700D9007B2E075F002A4FDACF08D43
:1032F700A3AE35AF3674036F4E700375A300AE35BA
:10330700AF367403BE00039F5013AC33AD34ED2FBB
:10331700FFEC3EFE90006D1252E8E0F5A3AE35AF2C
:1033270036EFB40B09EEB401057414125293AE359F
:10333700AF36EFB40B07EEB4010375F80D7835120D
:10334700531E0232B690003DE4F022753600753503
:103357000075F8099007B1E0FEA3E0FF7408BE000E
:103367001ED39F401A7E017F089007B1E0FCA3E0BF
:10337700FD1DBDFF011C1200038E338F34801F908B
:1033870007B1E0FEA3E0FF740812530E8F048E0509
:103397007E017F08CDCCCD1200038E338F34AE353E
:1033A700AF367411D39F74019E5003023482A2F981
:1033B700B3500302347FE5364535700375A3D2AEAB
:1033C70035AF3674016F4E700375A300AE35AF3657
:1033D70074026F4E700D9007B2E075F002A4FDAC59
:1033E700F08DA3AE35AF3674036F4E700375A3002F
:1033F700AE35AF3674046F4E700375A300AE35AFAC
:103407003674056F4E700375A300AE35AF3674067C
:103417006F4E700375A300AE35AF3674076F4E70ED
:103427000375A300AE35AF3674086F4E700375A3EE
:1034370000AE35AF367408BE00039F5016AC33ADEF
:1034470034ED2FFFEC3EFE9000681252E8E5A3F042
:1034570075A300AE35AF36EFB41009EEB4010574AD
:1034670014125293AE35AF36EFB41007EEB4010322
:1034770075F80D783512531E0233A522753600757F
:10348700350075F809AE35AF367417BE0004D39F03
:10349700500302355BA2F9B35003023558E53645B0
:1034A70035700375A3D2AE35AF3674016F4E700316
:1034B70075A300AE35AF3674026F4E700D9007B22C
:1034C700E075F002A4FDACF08DA3AE35AF36740302
:1034D7006F4E700375A300AE35AF3674046F4E7030
:1034E7000375A300AE35AF3674056F4E700375A331
:1034F70000AE35AF3674066F4E700375A300AE3558
:10350700AF3674076F4E700375A300AE35AF3674D0
:10351700086F4E700375A300AE35AF367408BE0052
:10352700039F500C9000511252E8E5A3F075A300D9
:10353700AE35AF3674166F4E70057414125293AED3
:1035470035AF3674166F4E700375F80D7835125314
:103557001E02348C2290003DE0B4AB02800302359A
:10356700F675360075350075F809AE35AF36741245
:10357700BE007CD39F4078A2F9B34070E53645354D
:10358700700375A382AE35AF3674016F4E70037545
:10359700A300AE35AF3674026F4E700D9007B2E0E0
:1035A70075F002A4FDACF08DA3AE35AF3674036F92
:1035B7004E700375A300AE35AF367403BE00039F8C
:1035C70050099000561252E8E0F5A3AE35AF3674B5
:1035D700116F4E70057414125293AE35AF367411D5
:1035E7006F4E700375F80D783512531E0235712230
:1035F700900046E4F074649007B1F8E4F0E8A3F0B3
:1036070012348374C89007B1F8E4F0E8A3F090008F
:103617005DE0B4371A90005AE0900051F090005BDB
:10362700E0900052F090005CE0900053F0804690EC
:1036370000467401F074659007B1F8E4F0E8A3F070
:1036470012348374C89007B1F8E4F0E8A3F090004F
:103657005DE0B4371A90005AE0900051F090005B9B
:10366700E0900052F090005CE0900053F080067408
:1036770002900046F0900047E4F074669007B1F8B6
:10368700E4F0E8A3F012348374C89007B1F8E4F0CB
:10369700E8A3F090005CE0B4371290005AE0900085
:1036A7004BF090005BE0900054F0807690004774F8
:1036B70001F074679007B1F8E4F0E8A3F0123483DF
:1036C70074C89007B1F8E4F0E8A3F090005CE0B4A8
:1036D700371290005AE090004BF090005BE09000AA
:1036E70054F0803E7402900047F074689007B1F878
:1036F700E4F0E8A3F012348374C89007B1F8E4F05B
:10370700E8A3F090005CE0B4371290005AE0900014
:103717004BF090005BE0900054F08006740390003B
:1037270047F022E55D2534FFAE3350010E9000715E
:103737001252E8E0F55EE55D2534FFAE3350010E29
:103747000FBF00010E9000711252E8E0F55F85652A
:1037570061E55EB55F05855E5D8041E55FD3955E9A
:10376700401DE55FC3955E8560F0A4FFAEF0E5619F
:103777008E048F05FF1252A3ED255EF55D801DE5D2
:103787005EC3955F8560F0A4FFAEF0E5618E048FA0
:1037970005FF1252A3EDF404255EF55D22E55FD324
:1037A700955E401DE55FC3955E8560F0A4FFAEF0B2
:1037B700E5618E048F05FF1252A3ED255EF55D804E
:1037C7001DE55EC3955F8560F0A4FFAEF0E5618EF1
:1037D700048F05FF1252A3EDF404255EF55D22E583
:1037E7003875F00484FF7E008F5DE53875F004843A
:1037F700ADF07C008D60756504753301753400E5A7
:103807005DC3943F500512372A80069001B0E0F55A
:103817005D855D53755200900042E075F020A4FF6E
:10382700AEF09000C2E08E048F05FF1252A38D5DAB
:103837009000AAE0D3953850030238EC9000CEE010
:10384700D395384010ED9001B11252F3E0F555755C
:1038570054000238E9900099E0D395384043E55D7C
:103867009001B11252F3E0F55EE55D9001D112527D
:10387700F3E0F55F9000CEE0F4042538F5609000A2
:1038870099E0FE9000CEE0F4042EF561E55EB55FA9
:1038970005855E5D80031237A4855D5575540080EC
:1038A70041E55D9001D11252F3E0F55EE55D9001CF
:1038B700F11252F3E0F55F900099E0F4042538F532
:1038C700609000AAE0FE900099E0F4042EF561E50F
:1038D7005EB55F05855E5D80031237A4855D55750E
:1038E70054000239939000D1E0D395385011E55D2B
:1038F7009002311252F3E0F5557554000239939056
:10390700009AE0D395385043E55D9002111252F3C7
:10391700E0F55EE55D9002311252F3E0F55F90004D
:103927009AE0F4042538F5609000D1E0FE90009A03
:10393700E0F4042EF561E55EB55F05855E5D800305
:103947001237A4855D557554008041E55D9001F1FE
:103957001252F3E0F55EE55D9002111252F3E0F5C5
:103967005F9000AAE0F4042538F56090009AE0FE25
:103977009000AAE0F4042EF561E55EB55F05855E6B
:103987005D80031237A4855D55755400229000E2CF
:10399700E0F562756511753302753400AE25AF2603
:1039A700E56275F00FA4FDACF0EDD39FEC9E4021CE
:1039B700E5628E048F05FF1252A3ED75F010A4FF88
:1039C700AEF0E53875F01184FD7C00ED2FF56380CE
:1039D7000EE53875F01184FF7E00EF24F0F563855E
:1039E700635DE53875F01184AFF07E008F601237A4
:1039F7002A855D64AE25AF269000E2E075F00FA43E
:103A0700FDACF0EDD39FEC9E402875330275341062
:103A170085635D12372A85645E855D5FAE25AF26B7
:103A2700E5628E048F05FF1252DC8D60856261129C
:103A370037A4855D537552007555647554002290FF
:103A470000E2E0F562756511753302753400AE2545
:103A5700AF26E56275F00FA4FDACF0EDD39FEC9EA9
:103A67004021E5628E048F05FF1252A3ED75F01019
:103A7700A4FFAEF0E53A75F01184FD7C00ED2FF55B
:103A870063800EE53A75F01184FF7E00EF24F0F5B0
:103A97006385635DE53A75F01184AFF07E008F6052
:103AA70012372A855D64AE25AF269000E2E075F0F7
:103AB7000FA4FDACF0EDD39FEC9E40287533027543
:103AC700341085635D12372A85645E855D5FAE2598
:103AD700AF26E5628E048F05FF1252DC8D6085628A
:103AE700611237A4855D537552009000ACE0B404B1
:103AF70053E53875F00484FF7E008F5DE53875F077
:103B07000484ADF07C008D607565047533017534F0
:103B170000E55DC3943F500512372A80069001B037
:103B2700E0F55DAE52AF53E55D1252C174648E0489
:103B37008F05FF1252A3AE52AF53EF2DFDEE3CFCA3
:103B47008C528D5375556475540022900077E0B4FC
:103B57000146E54075F00584FF7E008F5DE5407501
:103B6700F00584ADF07C008D6075650575330575CE
:103B77003400E55DC39417500512372A8006900577
:103B870088E0F55DAE54AF55E55D2FFF50010E742B
:103B97006412530E8E548F55900078E0B40146E5B9
:103BA7004175F00584FF7E008F5DE54175F0058462
:103BB700ADF07C008D60756505753305753448E596
:103BC7005DC39417500512372A80069005D0E0F59B
:103BD7005DAE54AF55E55D2FFF50010E746412536F
:103BE7000E8E548F55900087E0B40249E543C39485
:103BF7004175F00584FF7E008F5DE54375F0058410
:103C0700ADF07C008D60756505753306753400E58C
:103C17005DC39413500512372A8006900684E0F599
:103C27005DAE54AF55E55D2FFF50010E746412531E
:103C37000E8E548F559000C9E0B402028003023CF7
:103C4700F1E53875F01584FF7E008F5DE53875F076
:103C57001584ADF07C008D6075651575330375347B
:103C6700F4E55DC3940B500512372A800690047063
:103C7700E0F55DE55D75F0FFA4FFAEF09000CAE0EA
:103C87008E048F05FF1252A3ED90006BF0E53F7590
:103C9700F078A4FFAEF074FF8E048F05FF1252A3D5
:103CA7008C338D3474028C068D071252B38F5DAC42
:103CB70033AD347404FF1252DC8D607565047533BF
:103CC7000675346EE55DC3941D500512372A8006CC
:103CD7009006FCE0F55DAE54AF55E55D2FFF500152
:103CE7000E746412530E8E548F552290007FE0B4E9
:103CF70001179007B6E02555FFAE5450010E90000E
:103D0700D3E012530E8E548F5590007FE0B4031604
:103D1700A201B3B3501090006AE0C39405A825B878
:103D270000069526400280109000A1E02555FFAEC1
:103D37005450010E8E548F55900079E0B4020280E2
:103D470003023F1F90007CE0602FE540D3941E40A4
:103D570028900014E0FEA3E0FF9000B7E075F003A1
:103D6700A4FDACF0EFD39DEE9C400E9000DBE0A8E5
:103D770025B80005D395265003023F1F9000C4E0E5
:103D87008538F0A4FFAEF074051252C174071252C1
:103D9700B38E338F34900083E0A825B800049526AE
:103DA7005012900084E075F002A4FDACF0EFC39DC3
:103DB700EE9C4003023F1FE53875F00B84FF7E0041
:103DC7009006011252E8FEE0FFEE90007BE0FEEF66
:103DD7008E0088F0A4FFAEF074648E048F05FF1286
:103DE70052A38C338D34900042E075F018A4FFAED7
:103DF700F09000C2E08E048F05FF1252A38C068D4F
:103E0700079006191252E8AE33AF34E01252C1746C
:103E1700648E048F05FF1252A38C338D34E53EA8C0
:103E270033B80077D395344072E53EC39534FFE449
:103E37009533FE8E338F347428BE00039F500C7564
:103E47003428753300740D900045F0AE33AF3490CD
:103E5700007CE01252C174288E048F05FF1252A312
:103E67008C338D34AE52AF53740A8E048F05FF1214
:103E770052A38D068C07AC33AD34CFCECF120003DF
:103E8700740A8E048F05FF1252A38C338D34AE5201
:103E9700AF531253168E528F53807DE53EA833B829
:103EA700000495345072AE33AF34E53E12530E8E94
:103EB700338F347428BE00039F500C753428753334
:103EC70000740D900045F0AE33AF3490007CE012E3
:103ED70052C174288E048F05FF1252A38C338D3480
:103EE700AE52AF53740A8E048F05FF1252A38D068C
:103EF7008C07AC33AD34CFCECF120003740A8E04D7
:103F07008F05FF1252A38C338D34AE52AF53EF2D72
:103F1700FDEE3CFC8C528D5322AE52AF53AC54ADE8
:103F27005512000374648E048F05FF1252A38C523E
:103F37008D53900074E08C068D071252C174648E05
:103F4700048F05FF1252A38C528D53A2084017AE5F
:103F570025AF267405BE00039F5002D208E53AD369
:103F670094CC4002D2029000D6E0B402089000D868
:103F7700E0640160028017AE52AF53E5441252C1AC
:103F870074E78E048F05FF1252A38C528D53900055
:103F970096E05402601B90008DE0A825B80012D36C
:103FA7009526400DA208B3B35007E53AC3949A404B
:103FB700028028AE5BAF5C90008BE075F002A4FD39
:103FC700ACF0EF2DFDEE3CFC74022DFD50010CE52D
:103FD7003ABC0007D39D4003756901853A5C755B60
:103FE70000E56970030240769000E9E0C3956940F7
:103FF70070E54075F00584FF7E009005711252E868
:10400700E0F534753300AE33AF3490009BE01252C5
:10401700C174648E048F05FF1252A38C358D3690C0
:1040270000E9E004C395698C068D071252C1900020
:10403700E9E08E048F05FF1252A38C358D36900070
:104047008CE08C068D071252C1740A8E048F05FF0F
:104057001252A3AE52AF53EF2DFDEE3CFC8C528DA6
:104067005305699000E9E0C39569500375690090AD
:104077000096E05401601B90008AE0A825B8001262
:10408700D39526400DA208B3B35007E538C394CCA7
:1040970040028025900088E075F003A4FFAEF0E5AC
:1040A700662FFF50010E74032FFF50010EE538BE37
:1040B7000007D39F4003756A01853866E56A700378
:1040C7000241519000EAE0C3956A4070E54075F0FF
:1040D7000584FF7E009005711252E8E0F5347533D0
:1040E70000AE33AF3490009BE01252C174648E046B
:1040F7008F05FF1252A38C358D369000EAE004C37A
:10410700956A8C068D071252C19000EAE08E048FE3
:1041170005FF1252A38C358D36900089E08C068DF1
:10412700071252C1740A8E048F05FF1252A3AE52B2
:10413700AF53EF2DFDEE3CFC8C528D53056A90007A
:10414700EAE0C3956A5003756A0090009BE0A852A5
:10415700B800049553500990009BE0F55375520041
:10416700229000D7E0B401028003024273A208B391
:1041770050030242719000A2E0B40168AE52AF53FF
:10418700AC25AD26120003743C8E048F05FF125236
:10419700A39000B2E0BC00109D400D9000B4E0A8D1
:1041A70052B8000495535002D203AE52AF53AC2518
:1041B700AD26120003743C8E048F05FF1252A390A4
:1041C70000B2E0C3940ABC0015D39D40119000B41F
:1041D700E0C39405A852B80005D395535002800256
:1041E700C2038068AE52AF53AC25AD2612000374EC
:1041F700788E048F05FF1252A39000B2E0BC001026
:104207009D400D9000B4E0A852B8000495535004A7
:10421700D2038038AE52AF53AC25AD2612000374DB
:10422700788E048F05FF1252A39000B2E0C3940A60
:10423700BC0015D39D40119000B4E0C39405A8526B
:10424700B80005D3955350028002C203A203B340BE
:1042570019AE52AF539000B3E01252C174648E048A
:104267008F05FF1252A38C528D538002C203900018
:10427700D7E0B40258E53875F00884FF7E008F5DFB
:10428700E53875F00884ADF07C008D6075650875BC
:1042970033017534E0E55DC3943F500512372A803A
:1042A70006900270E0F55DE55D75F05EA4FFAEF087
:1042B700740A8E048F05FF1252A38C568D57740211
:1042C700BC000AD39D4006755702755600A200B37D
:1042D7004006A202B3B3500990001AE4F0A3F0809D
:1042E70024AE52AF537400D39F74019E400C9000CC
:1042F7001AE552F0A3E553F0800B74FF90001AF80B
:10430700E4F0E8A3F09000B9E0D394024006A208D5
:10431700B3B34002800DAE52AF5374021252C18E36
:10432700528F539000A2E0B4010DAE52AF53740206
:104337001252C18E528F53AE52AF53745E1252C196
:10434700740A8E048F05FF1252A38C528D53740288
:10435700BC000AD39D4006755302755200900018A1
:10436700E552F0A3E553F022900042E0900371126A
:1043770052F3E0F567756864900042E0FE9000AD87
:10438700E0D39E4037E53875F00884FF7E008F5DE7
:10439700E53875F00884ADF07C008D6075650875AB
:1043A7003303753496E55DC3941F500512372A8091
:1043B70006900426E0F55D855D688035E53875F083
:1043C7000884FF7E008F5DE53875F00884ADF07CCA
:1043D700008D607565087533037534B6E55DC39464
:1043E7001F500512372A8006900446E0F55D855D6B
:1043F70068229000E3E0F562756511753304753442
:1044070000AE25AF26E56275F00FA4FDACF0EDD345
:104417009FEC9E4021E5628E048F05FF1252A3EDAB
:1044270075F010A4FFAEF0E53875F01184FD7C003F
:10443700ED2FF563800EE53875F01184FF7E00EFF0
:1044470024F0F56385635DE53875F01184AFF07E80
:10445700008F6012372A855D64AE25AF269000E392
:10446700E075F00FA4FDACF0EDD39FEC9E402875EE
:10447700330475341085635D12372A85645E855D64
:104487005FAE25AF26E5628E048F05FF1252DC8DE5
:10449700608562611237A4855D6775686422900044
:1044A700E3E0F562756511753304753400AE25AF29
:1044B70026E56275F00FA4FDACF0EDD39FEC9E40AE
:1044C70021E5628E048F05FF1252A3ED75F010A44B
:1044D700FFAEF0E53A75F01184FD7C00ED2FF56332
:1044E700800EE53A75F01184FF7E00EF24F0F56346
:1044F70085635DE53A75F01184AFF07E008F601239
:10450700372A855D64AE25AF269000E3E075F00F8E
:10451700A4FDACF0EDD39FEC9E40287533047534B1
:104527001085635D12372A85645E855D5FAE25AFB2
:1045370026E5628E048F05FF1252DC8D608562616D
:104547001237A4855D677568649000DEE0B404796E
:10455700900042E0FE9000ADE0D39E4037E538750D
:10456700F00884FF7E008F5DE53875F00884ADF0B4
:104577007C008D60756508753303753496E55DC3FA
:10458700941F500512372A8006900426E0F55D85B2
:104597005D688035E53875F00884FF7E008F5DE53E
:1045A7003875F00884ADF07C008D6075650875334B
:1045B700037534B6E55DC3941F500512372A80068C
:1045C700900446E0F55D855D6822900077E0B401D0
:1045D7003BE54075F00584FF7E008F5DE54075F093
:1045E7000584ADF07C008D60756505753305753400
:1045F70018E55DC39417500512372A80069005A069
:10460700E0F55DE568255DC39464F568900078E0A2
:10461700B4013BE54175F00584FF7E008F5DE54100
:1046270075F00584ADF07C008D6075650575330503
:10463700753460E55DC39417500512372A800690DC
:1046470005E8E0F55DE568255DC39464F568E56711
:104657002568F55A90007FE0B402109007B5E02571
:104667005AFE9000D3E0F4042EF55A9000D6E0D31A
:1046770094014040E544C394E7501D74E7C3954453
:10468700FE9007B7E08E00F5F0E884FF7E008F5DAF
:10469700E55A255DF55A801CE544C394E7FE90076B
:1046A700B7E08E00F5F0E884FF7E008F5DE55AC322
:1046B700955DF55AA2084006E5672464F55AE55A60
:1046C700D394644009E55AC39464F55A8003755A34
:1046D700009000AFE0C3955A50069000AFE0F55A3E
:1046E70022D2009000C5E0A825B800049526503BCB
:1046F7009000C5E0A825B8000495265003755A0F09
:104707009000C5E004A825B8000495265003755A03
:104717000A9000C5E02402A825B800049526500594
:10472700755A05C2007409900045F07E017F00901C
:1047370000B5E01252C19000C4E08E048F05FF124D
:1047470052A3E538BC000CD39D4008C200740A9000
:104757000045F09000B6E0C39540500D9000C8E0CA
:10476700A825B80006952640028008C200740B9061
:104777000045F0A2004003755A0590007FE0B4039E
:1047870006A201B3B34002802B90006AE0C39405F0
:10479700A825B800049526500C9000A0E0F55A749F
:1047A7000C900045F090006AE0A825B80004952613
:1047B7005002C200855A45900071E0255AFE9000CC
:1047C70042E075F01E84FC7F00EE2CF55A22900023
:1047D70042E075F00584FF7E008F5D900042E07532
:1047E700F00584ADF07C008D607565057533037544
:1047F70034D69000C2E01475F00584FF7E00E55DB5
:10480700BE00039F500512372A800BE55D900447D1
:104817001252F3E0F55DE55D9007B8F09007B8E058
:10482700FE9000B1E0C39E50089000B1E09007B839
:10483700F022E54075F00584FF7E00900571125265
:10484700E8E0F56CE56CD394644010E56CC39464C0
:1048570075F00F84FF7E008F6C8003756C009000ED
:1048670094E0256CF56C229007ABE0FEA3E0FF74A3
:10487700041252B3E5381252C1740F8E048F05FF2C
:104887001252A39007A9ECF0A3EDF0900087E0B4D3
:104897000262E543C3944175F00584FF7E008F5D96
:1048A700E54375F00584ADF07C008D607565057591
:1048B7003306753414E55DC39417500512372A8003
:1048C70006900698E0F55D9007A9E0FEA3E0FF7467
:1048D7000A8E048F05FF1252A3E55D8C068D071221
:1048E70052C1740A8E048F05FF1252A39007A9ECD8
:1048F700F0A3EDF09007A9E0FEA3E0FF9007AFE07B
:10490700FCA3E0FDEDD39FEC9E400F9007AFE0F8CE
:10491700A3E09007A9C8F0A3C8F02290008EE0B4E6
:10492700010385265090008EE0B402129000C4E087
:104937008538F0A4FFAEF074081252B38F50900080
:104947008EE0B40303853A5090008EE0B4040385EB
:10495700405090008EE0B4050385415090008EE0F2
:10496700B4060385425090008EE0B4070385435098
:1049770090008EE0B4080385445090008EE0B4099F
:1049870003853F5090008EE0B40A03853E509000A7
:104997008EE0B40B0385455090008EE0B40C069072
:1049A700001BE0F55090008FE0FE900090E0D39E52
:1049B700404B90008EE0B40418900090E0C39550EF
:1049C7005002D20490008FE0D395504002C2048079
:1049D7002A90008FE0C395505009900090E0D3953E
:1049E7005050028002D20490008FE0D395505009B6
:1049F700900090E0C395505002C204802A90008F27
:104A0700E0D395504009900090E0C3955040028054
:104A170002C20490008FE0C395504009900090E0D7
:104A2700D395504002D20422900091E0B40103854F
:104A37002650900091E0B402129000C4E08538F04F
:104A4700A4FFAEF074081252B38F50900091E0B4F7
:104A57000303853A50900091E0B4040385405090D9
:104A67000091E0B40503854150900091E0B406033E
:104A7700854250900091E0B4070385435090009120
:104A8700E0B40803854450900091E0B40903853FE2
:104A970050900091E0B40A03853E50900091E0B435
:104AA7000B03854550900091E0B40C0690001BE085
:104AB700F550900092E0FE900093E0D39E40409026
:104AC7000092E0C395505009900093E0D395505061
:104AD700028002D206900092E0D3955050099000D0
:104AE70093E0C395505002C206900091E0B40109CB
:104AF7009000D0E0D3953A50028002C206802A90F7
:104B07000092E0D395504009900093E0C395504040
:104B1700028002C206900092E0C3955040099000BF
:104B270093E0D395504002D20622AE58AF5974F5A0
:104B3700D39F74019E4008785812531E024C4B7540
:104B47005901755800AE25AF26E56CBE000DD39F01
:104B570040099000A6E0D3956D40028023756D0053
:104B6700E56CC39526F5509000A9E0D3956B4008F6
:104B7700E56B2550F56B80069000A9E0F56B800288
:104B8700056D900082E0D3953A401CE538C395390E
:104B97004015AE25AF26E56CBE00039F5009900077
:104BA700A7E0D3956E4002806E9007B9E0A825B8BC
:104BB7000004952650037570009007B9E0A825B842
:104BC700000BD395264006E5269007B9F0E57070EF
:104BD70041E526C3956CF550E550D3940540037520
:104BE70050059000A8E0C3956B5007E550C3956B3F
:104BF70040028009E56BC39550F56B80069000A8CD
:104C0700E0F56B9000A8E0D3956B40069000A8E014
:104C1700F56B756E008002056EE570701690008268
:104C2700E0C3953A500DE56C2405A825B800069514
:104C3700264002800F900095E0F56B75700174783F
:104C47009007B9F022AE58AF5974E9D39F74039E09
:104C57004008785812531E024DEA755901755800DD
:104C6700756B32A223402A756B19900095E075F099
:104C770002A4FFAEF0E56DBE0006D39F4002D2232B
:104C8700056D75700374789007B9F0756F00024D64
:104C9700D9AE25AF26E56C6F4E7003024DD9E56C92
:104CA700BE000DD39F40099000A6E0D3956D40024A
:104CB700800F756D00E570C394035003756B198001
:104CC7000DE56CC39526F550E56D2550F56D900003
:104CD70082E0D3953A400E9007B9E0A825B80007BF
:104CE700D395264002800C056F900095E0B56F03C1
:104CF700757000E570B40306A208B3B34002800ADA
:104D0700056FE56FB43C03757002E570B402299036
:104D170007B9E0A825B8000ED395264009E52690E7
:104D270007B9F0756F00900082E0C3953A50097596
:104D37006F0074789007B9F0E570705A900082E0C0
:104D4700D3953A401CE538D395394015AE25AF26A3
:104D5700E56CBE00039F50099000A7E0D3956E4015
:104D6700028008756E00756B4B8028E526C3956C2D
:104D7700F550E550D394054003755005900082E047
:104D8700D3953A4008E56E2550F56E8006E56E240A
:104D970006F56E756F00E5707016900082E0C3959A
:104DA7003A500DE56C2405A825B800069526400263
:104DB7008003757001E570B40118756B19056F9064
:104DC7000095E0B56F06757002756F0074789007EF
:104DD700B9F0E56B75F00AA4FFAEF09007B3EEF0FB
:044DE700A3EFF02224
:0952F3002582F582500205832298
:0F008C0025E050020583258250020583F582226C
:10528200EF2F500205832582F582E5833E2EF583BA
:0152920022F9
:10530E00CFC39FFF50011E22C3EF9DFFEE9CFE22D6
:0952FC00E493F608740193F62214
:08531E000806B6000218062281
:0D52CF00A3E004F07006120049E004F02294
:0E003900A3E014F0B4FF06120049E014F02218
:0E52B300048007C3CE13CECF13CFD5E0F62272
:1051A100BC000FBE0008ED8FF084FFADF022E4FEDD
:1051B100FF22BE000DEF60FE54F0606F20E7030296
:1051C1005257EAC0E0EBC0E078017A0075F001EED9
:1051D10020E710EF25E0FFEE33FE0AC5F023C5F00E
:1051E10030E7F0EA5407F9096A7A007B00600108A8
:1051F100C3EC9E40167004ED9F4010ED9FFDEC9EA8
:10520100FCE5F0CA4ACA03F5F08005E5F003F5F0C4
:10521100C3EE13FEEF13FFD9D77908CACBCAD8D092
:10522100EAFEEBFFD0E0FBD0E0FA22EC8FF084FC49
:10523100ED54F045F0C48FF084FEEDC454F045F018
:10524100C48FF084FDEEC4FE54F02DFFEE540F3CEC
:10525100FEADF07C0022790078008FF0EC7E082012
:10526100E70DC3CD33CD33C933C9C833C8DEF084AC
:1052710049F9E5F08FF0BE00E6FD7C00E9FFE8FEAC
:01528100220A
:0E52C100F88FF0A4FFE5F0CE88F0A42EFE22B8
:10000300EF8DF0A4F9A8F0EF8CF0A428F8EE8DF0B2
:06001300A428FEE9FF2213
:10529300600D782B02529D007830D8FED5E0F822BD
:1052A300EEC0E07E001251A1EFFDEEFCD0E0FE2245
:0C52DC00EEC0E07E001251A1D0E0FE22E6
:03001B0002001EC2
:0300530002005652
:03009B00020071EF
:03000000025305A3
:0953050075817175D0000206B833
:0B52E800E5822FF582E5833EF583226E
:0A0049000582D5820215831582227C
:10001E00C0E0C0F0C083C082C0D075D000120643CD
:0B002E00D0D0D082D083D0F0D0E032E0
:10005600C0E0C0F0C083C082C0D075D00012064692
:10006600D0D0D082D083D0F0D0E032C0E0C0F0C093
:1000760083C082C0D075D000120655D0D0D082D0B1
:0600860083D0F0D0E0324F
:00000001FF
